:103800000C94381C0C94551C0C94551C0C94551C91
:103810000C94551C0C94551C0C94551C0C94551C64
:103820000C94551C0C94551C0C94551C0C94551C54
:103830000C94551C0C94551C0C94551C0C94551C44
:103840000C94551C0C94551C0C94551C0C94551C34
:103850000C94551C0C94551C0C94551C0C94551C24
:103860000C94551C0C94551C0C94551C0C94551C14
:1038700011241FBECFEFD4E0DEBFCDBF11E0A0E02A
:10388000B1E0E8EDFDE302C005900D92A030B10774
:10389000D9F711E0A0E0B1E001C01D92A030B1075E
:1038A000E1F70E942D1D0C94EB1E0C94001C0F934D
:1038B0001F93CF93DF938C01EA01653489F48881EB
:1038C00099818EBB292F33272FBB0196998388833B
:1038D000E09A8DB30E94E11E0150104081F721C093
:1038E0006634F9F488819981880F991F99838883B8
:1038F000E881F981E4918E2F0E94E11EE881F9812F
:103900003196E4918E2F0E94E11E88819981029662
:10391000998388830250104059F79695879599832B
:103920008883DF91CF911F910F910895AF92BF923D
:10393000CF92DF92EF92FF920F931F93CF93DF937B
:10394000CDB7DEB7C058D0400FB6F894DEBF0FBE7B
:10395000CDBF5C016A01653471F500E010E008C07C
:103960000E94E61EFE01E00FF11F81830F5F1F4FD3
:103970000A151B05A9F707B600FCFDCF40E050E093
:10398000FE0114C0D6012D913C912EBB832F9927A7
:103990008FBB80818DBBE29AE19AE199FECF2F5FC8
:1039A0003F4FD6012D933C934F5F5F4F31964A15A1
:1039B0005B0541F73EC0663419F08FE390E03BC0F1
:1039C000FA01E080F180EE0CFF1CF182E0820E949F
:1039D000E61E082F11270E94E61ED6012D913C916C
:1039E00041E09927982F8827082B192B0801F90106
:1039F00040935700E89511242E5F3F4FF601318325
:103A000020838EEF9FEFA80EB91EA114B104F9F622
:103A100085E0F70180935700E89507B600FCFDCFDD
:103A200081E180935700E89536952795D6012D932F
:103A30003C938DE090E0C058DF4F0FB6F894DEBFA6
:103A40000FBECDBFDF91CF911F910F91FF90EF90EF
:103A5000DF90CF90BF90AF900895EF92FF920F93B9
:103A60001F93CF93DF93CDB7DEB722970FB6F894AD
:103A7000DEBF0FBECDBF1BBA8FE38ABB80E182BB26
:103A8000949A0E94DC1EDD9A84997FC1D89A0E9484
:103A9000E61E282F8BB398E089278BBB213611F4C3
:103AA00089E570C1213471F40E94E61E082F0E943E
:103AB000E61E1127102F00279927082B192B1A8390
:103AC000098333C1253689F480E090E023E007B60E
:103AD00000FCFDCFFC0120935700E89580589F4FD4
:103AE00038E38030930798F39DC0223641F489E58E
:103AF0000E94E11E80E00E94E11E80E843C1223462
:103B0000A9F40E94E61E082F0E94E61E1127F02E3F
:103B1000EE249927E82AF92A0E94E61EAE014F5F9B
:103B20005F4F682FC7010E94961C2CC12736A9F44D
:103B30000E94E61E082F0E94E61E1127F02EEE249A
:103B40009927E82AF92A0E94E61EAE014F5F5F4FCF
:103B5000682FC7010E94571C9ACF2235B9F407B6C7
:103B600000FCFDCF81E180935700E895E981FA815F
:103B7000EE0FFF1F3196E4918E2F0E94E11EE98126
:103B8000FA81EE0FFF1FE4918E2F59C0233629F4DE
:103B90000E94E61EE82EFF24C8C02334B9F40E9418
:103BA000E61E9927982F8827E82AF92A07B600FCED
:103BB000FDCF89819A8141E09C01220F331F0701CB
:103BC000F90140935700E89511242BC02D36A9F434
:103BD00029813A818CE12030380720F08FE30E9460
:103BE000E11EA3C007B600FCFDCF85E0220F331F06
:103BF000F90180935700E89598C02434B1F407B6D2
:103C000000FCFDCF89819A818EBB892F99278FBBBC
:103C10000E94E61E8DBBE29AE19AE199FECF89816E
:103C20009A8101969A83898380C0243681F48981A0
:103C30009A818EBB892F99278FBBE09A8DB30E9402
:103C4000E11E89819A8101969A83898320CF2C363F
:103C500069F407B600FCFDCF0E94E61E99E0E1E0A2
:103C6000F0E0082E90935700E8955FC0223751F49A
:103C700007B600FCFDCF89E0E1E0F0E0809357005B
:103C8000849180C0263451F407B600FCFDCF89E052
:103C9000E0E0F0E080935700849174C02E3451F43A
:103CA00007B600FCFDCF89E0E3E0F0E08093570029
:103CB000849168C0213551F407B600FCFDCF89E03E
:103CC000E2E0F0E08093570084915CC0203569F118
:103CD0002C3459F1253471F407B600FCFDCF81E195
:103CE00080935700E8958DE00E94E11EE0E0F0E04F
:103CF0000995CDCE203711F483E544C0243729F44B
:103D000083E60E94E11E80E03DC0283721F40E9436
:103D1000E61EDC9A0AC0293721F40E94E61EDC98D0
:103D200004C0243521F40E94E61E8DE02BC023350B
:103D3000A1F481E40E94E11E86E50E94E11E82E575
:103D40000E94E11E82E40E94E11E8FE40E94E11EB7
:103D50008FE40E94E11E84E515C0263529F481E335
:103D60000E94E11E85E30EC0233741F484E00E94E7
:103D7000E11E84E90E94E11E8EE104C02B3109F4AA
:103D800086CE8FE30E94E11E82CE07B600FCFDCFF7
:103D900081E180935700E895E0E0F0E009952296F4
:103DA0000FB6F894DEBF0FBECDBFDF91CF911F914C
:103DB0000F91FF90EF90089583E389B988E18AB964
:103DC00008958CB95E9BFECF5E9A08955F9BFECFEF
:083DD0008CB199270895FFCF83
:0400000300003800C1
:00000001FF
